:100000008FEF1BF000000000D6EF1AF00000000098
:0C001000000000000000000060EF1BF08A
:0E001C00ACB202D00000FCD72EC3ADFF120024
:0C002A0072B201D0FDD72EC373FF12008C
:100036006DB409D01F0E6B14016E0150000A03E166
:0A004600010E006E01D0006A1200E6
:10005000C7B409D01F0EC514016E0150000A03E198
:0A006000010E006E01D0006A1200CC
:10006A00F250026EF29E0500FF6A0150FE6E0050C9
:08007A00FD6E02BEF28E1200C1
:0A008200000E9EBA010E006E12007F
:10008C00AECF01F0ABA202D0AB98AB8801C000F0B0
:02009C00120050
:10009E0054C02AF355C02BF356C02CF357C02DF382
:1000AE000301286B296B2951120802E128518E0891
:1000BE0008E3BADF005201E004D00301284B292BDC
:1000CE00F2D70301120E295D02E18F0E285D03E3C4
:1000DE007B0E006E24D06B806BA020D05450551038
:1000EE00561057101AE02A512B112C112D110EE11A
:1000FE00C8C1E1FFC9C1E2FF050EE66EC6C100F040
:10010E00C7C101F0ABDF010E006E09D0010E030175
:10011E002A5F000E2B5B2C5B2D5BDED7006A120074
:0A012E00000EA4BA010E006E1200CC
:1001380074CF01F071A202D07198718801C000F0EB
:020148001200A3
:10014A0050C02AF351C02BF352C02CF353C02DF3E5
:10015A000301286B296B2951120802E128518E08E4
:10016A0008E371DF005201E004D00301284B292B78
:10017A00F2D70301120E295D02E18F0E285D03E317
:10018A007B0E006E24D0C580C5A020D050505110DF
:10019A00521053101AE02A512B112C112D110EE175
:1001AA00CCC1E1FFCDC1E2FF050EE66ECAC100F087
:1001BA00CBC101F055DF010E006E09D0010E03011B
:1001CA002A5F000E2B5B2C5B2D5BDED7006A1200C8
:0A01DA00000EACB2010E006E120020
:0A01E400000E72B2010E006E120050
:0E01EE00026A016A006A086A036A000E1200C3
:1001FC000B820BAE08EF01F003680268016800681F
:08020C000A360232FF0E120057
:0A02140000000000000000001200CE
:0A021E001D0E0D6E0D2EFED712000E
:080228000AAE029E000E120056
:100230000B840BAE23EF01F0010E036E026A016A1C
:0A024000006A0A360232FF0E1200B7
:0C024A0001C200F002C201F00BDF120044
:1002560054C022F355C023F356C024F357C025F3E8
:100266006B826BA21FD0545055105610571019E0D0
:10027600030122512311241125110CE1C8C1E1FF0C
:10028600C9C1E2FF060EE66EC6C100F0C7C101F0A5
:10029600E9DE08D0010E0301225F000E235B245B1A
:0602A600255BDFD712000A
:1002AC00800E0301236F221F235316E023512215C6
:1002BC00016E0152010ED8A4000E006E00B002D0E7
:1002CC00829A01D0828AA0DF9FDF8286A2DF82968B
:0A02DC00A0DF2333239FE8D71200B0
:1002E60054C024F355C025F356C026F357C027F350
:1002F600A49E6B86A4BE1FD054505510561057109E
:1003060019E0030124512511261127110CE1C8C15A
:10031600E1FFC9C1E2FF030EE66EC6C100F0C7C128
:1003260001F0A0DE08D0010E0301245F000E255B5C
:10033600265B275BDFD703016FCF23F32251000A29
:1003460002E16B8A01D06B9AA49E6B8854C024F399
:1003560055C025F356C026F357C027F3A4BE1FD0B9
:10036600545055105610571019E003012451251109
:10037600261127110CE1C8C1E1FFC9C1E2FF030E36
:10038600E66EC6C100F0C7C101F06CDE08D0010EF2
:100396000301245F000E255B265B275BDFD723C3A3
:0403A60000F0120051
:0403AA006B8412004E
:1003AE00A49E22C36FFF54C023F355C024F356C03E
:1003BE0025F357C026F36DA421D054505510561076
:1003CE0057101BE0030123512411251126110EE1B4
:1003DE00C8C1E1FFC9C1E2FF040EE66EC6C100F05E
:1003EE00C7C101F03BDE010E006E3AD0010E0301D3
:1003FE00235F000E245B255B265BDDD754C023F301
:10040E0055C024F356C025F357C026F3A4BE21D001
:10041E0054505510561057101BE003012351241150
:10042E00251126110EE1C8C1E1FFC9C1E2FF040E7C
:10043E00E66EC6C100F0C7C101F010DE010E006EFF
:10044E000FD0010E0301235F000E245B255B265B9C
:10045E00DDD76BBC02D0006A03D06B84020E006E37
:02046E0012007A
:100470000CB07AEF02F00CA220EF03F00E6A000E2F
:10048000026491EF02F0F00E0214D8A45CEF02F0C7
:10049000023A01380F0B02260138F00B016E0038CA
:1004A0000F0B01260038F00B006E08380F0B0026EA
:1004B0000838F00B086E0E84D89002BE75EF02F07B
:1004C00008360036013602360E2A02BE75EF02F0FB
:1004D00008360036013602360E2A02BE75EF02F0EB
:1004E00008360036013602360E2A0E50036416EF27
:1004F00003F0035E0BBC08AE1BEF03F0D880800E48
:1005000008640030000E002201220222D8A01BEF56
:1005100003F0023201320032034A20EF03F01BEFF6
:1005200003F001C002F000C001F008C000F0086A4A
:10053000000E0E860264C8EF02F0F00E0214D8A47A
:10054000B0EF02F0023A01380F0B02260138F00B2F
:10055000016E00380F0B01260038F00B006E0E8480
:10056000D89002BE75EF02F00036013602360E2A30
:1005700002BE75EF02F00036013602360E2A02BEC8
:1005800075EF02F00036013602360E2A75EF02F0E2
:1005900001C002F000C001F0006A000E0E960E8845
:1005A0000264F5EF02F0F00E0214D8A4E0EF02F0BE
:1005B000023A01380F0B02260138F00B016E0E844F
:1005C000D89002BE75EF02F0013602360E2A02BE46
:1005D00075EF02F0013602360E2A02BE75EF02F008
:1005E000013602360E2A75EF02F001C002F0016AF0
:1005F000000E0E86026425EF03F0F00E0214D8A45C
:1006000004EF03F0023A0E84D89002BE75EF02F0B8
:1006100002360E2A02BE75EF02F002360E2A02BE24
:1006200075EF02F002360E2A75EF02F0010E0C6E25
:10063000FFDD28EF03F0020E0C6EF6DD28EF03F06D
:10064000040E0C6EDBDD28EF03F0080E0C6ECFDD20
:02065000120096
:100652000450085E0550D8A0053C095E0650D8A09B
:10066200063C0A5E0750D8A0073C0B5E0336070E15
:100672000C6E0334083609360A360B36045003A0D2
:100682000ED0085E0550D8A0053C095E0650D8A0E1
:10069200063C0A5E0750D8A0073C0B5E0DD0082628
:1006A2000550D8B0053C09260650D8B0063C0A26AB
:1006B2000750D8B0073C0B2603360C2EDAD702348B
:1006C200083609360A360B36045003A00ED0085EEF
:1006D2000550D8A0053C095E0650D8A0063C0A5E2B
:1006E2000750D8A0073C0B5E0DD008260550D8B0A5
:1006F200053C09260650D8B0063C0A260750D8B059
:10070200073C0B260236070E0C6E023408360936F9
:100712000A360B36045002A00ED0085E0550D8A04F
:10072200053C095E0650D8A0063C0A5E0750D8A0D8
:10073200073C0B5E0DD008260550D8B0053C0926B3
:100742000650D8B0063C0A260750D8B0073C0B2604
:1007520002360C2EDAD70134083609360A360B3641
:10076200045002A00ED0085E0550D8A0053C095ED8
:100772000650D8A0063C0A5E0750D8A0073C0B5E84
:100782000DD008260550D8B0053C09260650D8B031
:10079200063C0A260750D8B0073C0B260136070E46
:1007A2000C6E0134083609360A360B36045001A0A5
:1007B2000ED0085E0550D8A0053C095E0650D8A0B0
:1007C200063C0A5E0750D8A0073C0B5E0DD00826F7
:1007D2000550D8B0053C09260650D8B0063C0A267A
:1007E2000750D8B0073C0B2601360C2EDAD700345E
:1007F200083609360A360B36045001A00ED0085EC0
:100802000550D8A0053C095E0650D8A0063C0A5EF9
:100812000750D8A0073C0B5E0DD008260550D8B073
:10082200053C09260650D8B0063C0A260750D8B027
:10083200073C0B260036070E0C6E003408360936CC
:100842000A360B36045000A00ED0085E0550D8A020
:10085200053C095E0650D8A0063C0A5E0750D8A0A7
:10086200073C0B5E0DD008260550D8B0053C092682
:100872000650D8B0063C0A260750D8B0073C0B26D3
:1008820000360C2EDAD700B00ED0045008260550E0
:10089200D8B0053C09260650D8B0063C0A260750B7
:0808A200D8B0073C0B26120040
:1008AA00CFDCD00E0301226F7DDD1DC322F37ADD7A
:1008BA001EC322F377DDCADC03011F6B206B800E97
:1008CA002019006E800E005C02E1030E1F5D0EE22D
:1008DA00D00E226F67DD0050010A03E14FEC00F0F1
:1008EA0001D004D003011F4B202BE9D759DD120098
:1008FA000B6A0A6A096A00500402F4CF09F0F3CFBE
:10090A0008F001500502F4CF0BF0F3CF0AF00050C3
:10091A000502F3500926F4500A22E86A0B22015014
:10092A000402F3500926F4500A22E86A0B2208C08E
:10093A0000F009C001F00AC002F00BC003F0120077
:10094A00086A080E0C6E003408360450085ED8B0E7
:0E095A0002D00826D89000360C2EF5D71200D9
:100968000B6A0A6A096A086A0E6A03340836045070
:10097800085E0550D8A0053C095E0650D8A0063C84
:100988000A5E0750D8A0073C0B5EE86AD8A0010EA3
:100998000E5E0336070E0C6E0334083609360A3627
:1009A8000B360E36045003A012D0085E0550D8A0AE
:1009B800053C095E0650D8A0063C0A5E0750D8A040
:1009C800073C0B5EE86AD8A0010E0E5E11D008261F
:1009D8000550D8B0053C09260650D8B0063C0A2672
:1009E8000750D8B0073C0B26E86AD8B0010E0E268F
:1009F80003360C2ED1D70234083609360A360B36A0
:100A08000E36045003A012D0085E0550D8A0053C4D
:100A1800095E0650D8A0063C0A5E0750D8A0073CDD
:100A28000B5EE86AD8A0010E0E5E11D008260550AC
:100A3800D8B0053C09260650D8B0063C0A2607500F
:100A4800D8B0073C0B26E86AD8B0010E0E2602364D
:100A5800070E0C6E0234083609360A360B360E3687
:100A6800045002A012D0085E0550D8A0053C095ECB
:100A78000650D8A0063C0A5E0750D8A0073C0B5E7B
:100A8800E86AD8A0010E0E5E11D008260550D8B02D
:100A9800053C09260650D8B0063C0A260750D8B0AF
:100AA800073C0B26E86AD8B0010E0E2602360C2E3B
:100AB800D1D70134083609360A360B360E360450BB
:100AC80002A012D0085E0550D8A0053C095E065069
:100AD800D8A0063C0A5E0750D8A0073C0B5EE86A1F
:100AE800D8A0010E0E5E11D008260550D8B0053CDE
:100AF80009260650D8B0063C0A260750D8B0073C4D
:100B08000B26E86AD8B0010E0E260136070E0C6EC9
:100B18000134083609360A360B360E36045001A061
:100B280012D0085E0550D8A0053C095E0650D8A032
:100B3800063C0A5E0750D8A0073C0B5EE86AD8A0BE
:100B4800010E0E5E11D008260550D8B0053C0926C6
:100B58000650D8B0063C0A260750D8B0073C0B26EA
:100B6800E86AD8B0010E0E2601360C2ED1D7003413
:100B7800083609360A360B360E36045001A012D054
:100B8800085E0550D8A0053C095E0650D8A0063C72
:100B98000A5E0750D8A0073C0B5EE86AD8A0010E91
:100BA8000E5E11D008260550D8B0053C092606501F
:100BB800D8B0063C0A260750D8B0073C0B26E86A8E
:100BC800D8B0010E0E260036070E0C6E003408361B
:100BD80009360A360B360E36045000A012D0085ECD
:100BE8000550D8A0053C095E0650D8A0063C0A5E10
:100BF8000750D8A0073C0B5EE86AD8A0010E0E5E2D
:100C080011D008260550D8B0053C09260650D8B0A2
:100C1800063C0A260750D8B0073C0B26E86AD8B02D
:100C2800010E0E2600360C2ED1D700B00ED004507F
:100C380008260550D8B0053C09260650D8B0063C11
:0C0C48000A260750D8B0073C0B2612000B
:100C54008B901DC322F356EC01F01EC322F356EC15
:100C640001F01DC322F356EC01F01FC322F356EC2E
:100C740001F01DC322F356EC01F020C322F356EC1D
:100C840001F01DC322F356EC01F021C322F356EC0C
:060C940001F08B8012004C
:100C9A004FEC00F0D00E0301226FD7EC01F01DC318
:100CAA0022F3D7EC01F04FEC00F0D10E0301226FD2
:100CBA00D7EC01F00301226B73EC01F000C009F2DA
:100CCA00000E02010A6FD5EC01F009C200F0120011
:100CDA000B1E0A1E091E081E082AD8B4092AD8B4EF
:080CEA000A2AD8B40B2A1200FB
:100CF200086A096A100E0C6E01340836093604506F
:100D0200085E0550D8A0053C095ED8B007D0045053
:100D120008260550D8B0053C0926D8900036013681
:060D22000C2EEAD71200BE
:100D28000B800BAEA0EF06F0026A0AAEFF0E026E51
:0C0D3800016E006E0A360232FF0E12003F
:100D4400025006180E6E086A096A0B6A035007649B
:100D540095EF07F006500A6E068E028E03500B6E56
:100D64000750036E000E0B64E5EF06F00B50075EB0
:100D7400D8B486EF07F0070E076454EF07F0075E58
:100D840000C008F001C000F002C001F0026A074E82
:100D940086EF07F0076429EF07F0075E00C008F04C
:100DA40001C000F0016A074E86EF07F0076407EF01
:100DB40007F0075E00C008F0006A074E86EF07F0F0
:100DC4000764EEEF06F00AC002F005C001F004C0AB
:100DD40000F0086AB2EF08F0030E0764F9EF06F0BA
:100DE400075E08380F0B086E074E86EF07F0D890A1
:100DF4000832074E86EF07F0D8900832074E86EF88
:100E040007F0D890083286EF07F0030E076418EF56
:100E140007F0075E08380F0B086E0038F00B082641
:100E240000380F0B006E074E86EF07F0D8900032A3
:100E34000832074E86EF07F0D89000320832074E8A
:100E440086EF07F0D8900032083286EF07F0030EE1
:100E5400076440EF07F0075E08380F0B086E003890
:100E6400F00B082600380F0B006E0138F00B00263B
:100E740001380F0B016E074E86EF07F0D890013250
:100E840000320832074E86EF07F0D8900132003264
:100E94000832074E86EF07F0D8900132003208324C
:100EA40086EF07F0030E076471EF07F0075E08385A
:100EB4000F0B086E0038F00B082600380F0B006E7D
:100EC4000138F00B002601380F0B016E0238F00BCD
:100ED400012602380F0B026E074E86EF07F0D890FA
:100EE4000232013200320832074E86EF07F0D89002
:100EF4000232013200320832074E86EF07F0D890F2
:100F04000232013200320832096A000E0EAE7AEF64
:100F140008F0081E001E011E021E082A00220122DB
:100F240002227AEF08F00750D8A49BEF07F0B2EF43
:100F340008F0096A02C00AF0028E068E0750035CAC
:100F4400076ED8B46DEF08F0070E07643BEF08F0A6
:100F5400075E0450096E0550046E0650056E066A5D
:100F6400074E6DEF08F0070E076410EF08F0075EF8
:100F74000450096E0550046E056A074E6DEF08F0C3
:100F8400070E0764EEEF07F0075E0450096E046A6B
:100F9400074E6DEF08F0070E0764D5EF07F00AC09F
:100FA40002F0B2EF08F0030E0764E0EF07F0075E0B
:100FB40009380F0B096E074E6DEF08F0D89009320F
:100FC400074E6DEF08F0D8900932074E6DEF08F028
:100FD400D89009326DEF08F0030E0764FFEF07F0B5
:100FE400075E09380F0B096E0438F00B0926043824
:100FF4000F0B046E074E6DEF08F0D89004320932DF
:10100400074E6DEF08F0D89004320932074E6DEFA9
:1010140008F0D890043209326DEF08F0030E07642B
:1010240027EF08F0075E09380F0B096E0438F00B40
:10103400092604380F0B046E0538F00B0426053816
:101044000F0B056E074E6DEF08F0D8900532043291
:101054000932074E6DEF08F0D89005320432093298
:10106400074E6DEF08F0D8900532043209326DEF67
:1010740008F0030E076458EF08F0075E09380F0BF9
:10108400096E0438F00B092604380F0B046E05387A
:10109400F00B042605380F0B056E0638F00B0526F9
:1010A40006380F0B066E074E6DEF08F0D890063227
:1010B400053204320932074E6DEF08F0D89006323B
:1010C400053204320932074E6DEF08F0D89006322B
:1010D400053204320932086A000E0EAE7AEF08F0C7
:1010E400091E041E051E061E092A042205220622C4
:1010F40009500826045000220550012206500222FD
:101104000EBE91EF08F0D8A0A0EF08F00232013231
:1011140000320832033EA0EF08F0ACEF08F0D8B07C
:10112400A6EF08F0000E081E001E011E021E082A6B
:101134000022012202220A7EA6EF08F0010E0C6EA4
:1011440038EC02F0B4EF08F0020E0C6E38EC02F04A
:10115400B4EF08F0040E0C6EFEEC00F0B4EF08F0EF
:06116400000E0C6E1200EB
:10116A000C6A0E6A0250D8A4CEEF08F001C002F051
:10117A0000C001F0006A0E860250D8A4CEEF08F033
:10118A0001C002F0016A0E960E880250D8B4E0EF50
:10119A0008F00E50035ED8A4D8A0E6EF08F0D89065
:1011AA0002BEECEF08F0003601360236032ED5EF08
:1011BA0008F0E6EF08F0010E0C6EF7EC00F0F0EF25
:1011CA0008F0020E0C6E18EC01F0F0EF08F0040EB5
:0811DA000C6E14EC01F0120090
:0811E2000B6A0B86FF0E1200E0
:1011EA0003011D51390806E3300E1D5D03E3010EAC
:0811FA00006E01D0006A120032
:101202000FC3F6FF10C3F7FF11C3F8FF0900F5CFB4
:1012120000F0005212E00FC3F6FF10C3F7FF11C334
:10122200F8FF0900F5CF2EF30EEC00F0010E0301DA
:0C1232000F27000E10231123E3D7120039
:10123E000301116B0FC3E9FF10C3EAFFEECF00F3FA
:10124E000051000A0FE000C32EF30EEC00F0030174
:10125E00112B11510F25E96E000E1021EA6EEECF03
:06126E0000F3EED71200B0
:06127400067E66DD12009B
:10127A000A6A0350D8A40A800750D8A40A820A50DE
:10128A00D8B4A0EF09F0030AD8B459EF09F00AB0AC
:10129A0054EF09F006AE9EEF09F09CEF09F002AE9A
:1012AA009CEF09F09EEF09F00250800B0A6E029E35
:1012BA000650800B069E0A18D8B46AEF09F00A5045
:1012CA00D8B49CEF09F09EEF09F00750035CD8B43C
:1012DA0074EF09F0D8A090EF09F096EF09F00650E4
:1012EA00025CD8B47EEF09F0D8A090EF09F096EF2F
:1012FA0009F00550015CD8B488EF09F0D8A090EF46
:10130A0009F096EF09F00450005CD8B4A0EF09F098
:10131A00D8B096EF09F00A52D8B49EEF09F09CEFC4
:10132A0009F00A52D8B49CEF09F09EEF09F0D88070
:0E133A001200D8901200D880D8841200120041
:10134800086A096A000E0762036429EF0AF002506E
:1013580006180A6E075003267E0ED8A0BAEF09F0C9
:10136800035ED8B02EEF0AF0BEEF09F0035ED8A0F6
:1013780033EF0AF0028E068E02C00EF001C00BF0A9
:1013880000C00DF000500402F4CF0CF0015005022B
:10139800F4CF00F0F3CF08F00402F3500C26F45019
:1013A8000822000E00220D500502F3500C26F450BE
:1013B8000822000E002202500402F3500826F450BE
:1013C800002202500502016A000E0122F350002695
:1013D800F45001220D500602F3500826F450002262
:1013E800026A000E012202220B500602F350002668
:1013F800F4500122000E02220E500602F35001267C
:10140800F450022202BE11EF0AF008360036013607
:1014180002360306D8B433EF0AF024EF0AF0D88076
:10142800800E08640030000E002201220222D8A09B
:1014380024EF0AF0023201320032034A2EEF0AF09A
:101448000AAE029E000E36EF0AF0010EF7EC00F02D
:1014580036EF0AF0020EFEEC00F036EF0AF0040E4A
:0614680018EC01F0120077
:10146E000FC3E9FF10C3EAFFEECF11F3000E030125
:10147E00126F000E126F000E121902E1200E1119DA
:10148E0007E0000E121902E1090E111901E003D056
:10149E000F4B102BE5D7136B146B156B166B000EE1
:1014AE00121902E12D0E111905E1154B162B0F4BDA
:1014BE00102B08D0000E121902E12B0E111902E1A9
:1014CE000F4B102B0FC3E9FF10C3EAFFEECF11F342
:1014DE00000E126F000E126F11C31DF37FDE00524D
:1014EE0019E013C300F014C301F00A0E046E000ECF
:1014FE00056E7DEC04F0300E115D026E000E125979
:10150E00036E02500024136F03500120146F0F4B13
:10151E00102BD8D71551161108E013510008006E84
:10152E0014C301F0000E015604D013C300F014C30F
:04153E0001F01200A6
:101542004FEC00F0D00E0301226FD7EC01F0030143
:10155200226BD7EC01F0800E03010F25006E000E06
:101562001021016E00C022F3D7EC01F011C322F367
:10157200D7EC01F013C322F3D7EC01F015C322F329
:10158200D7EC01F017C322F3D7EC01F019C322F311
:10159200D7EC01F01BC322F3D7EC01F0D5EC01F03C
:1015A2004FEC00F0340E0C6EF10E0D6E0D2EFED7C8
:1015B2000C2EFCD700000000D00E0301226FD7ECE6
:1015C20001F00301226BD7EC01F00301226BD7EC8F
:0815D20001F0D5EC01F012005C
:1015DA000450000A12E10550000A0FE10650000A01
:1015EA000CE10750000A09E1FF0E006EFF0E016EC2
:1015FA007F0E026EFF0E036EA7D0086A096A0750B3
:10160A00D8B498EF0BF00350D8B49CEF0BF002500B
:10161A0006180A6E028E068E0E6A02C008F001C013
:10162A000CF000C00DF004500D5E0550D8A0053C2A
:10163A000C5E0650D8A0063C085E086A0C6A0D6A61
:10164A00D8A02FEF0BF0D8900232013200320832C4
:10165A00010E0E6E0750035ED8A03CEF0BF07E0E13
:10166A000E240326D8B0A1EF0BF042EF0BF07E0E4A
:10167A000E240326D8A0A6EF0BF0180E0B6E0D361B
:10168A000C3608360036013602360E360450005E35
:10169A000550D8A0053C015E0650D8A0063C025E63
:1016AA0006340E120EA05DEF0BF00D8068EF0BF002
:1016BA00045000260550D8B0053C01260650D8B083
:1016CA00062802260D900B2E44EF0BF08EEF0BF03E
:1016DA00D8900036013602360E360450005E0550A8
:1016EA00D8A0053C015E0650D8A0063C025E06342E
:1016FA000E10010B0D26D8B00C2AD8B4082AD8A48B
:10170A008EEF0BF008320C320D32032AD8B4A1EF57
:10171A000BF00AAE089E0850026E0C50016E0D5076
:10172A00006EA9EF0BF0010E57DDA9EF0BF0020EC8
:10173A00F7EC00F0A9EF0BF0040EFEEC00F0A9EFB5
:0A174A000BF0080E18EC01F012007D
:101754000FC3E9FF10C3EAFFEE500301111905E1BD
:101764000FC300F010C301F010D00FC300F010C37A
:1017740001F00F4B102B00C0E9FF01C0EAFFEECFD0
:0C17840000F00052E5E1006A016A12006A
:1017900003010F6B005109081DE20A0E046E00C31D
:1017A00000F0A5EC04F000C00FF300C00FF30F37FA
:1017B0000F910F370F910F370F910F370F910A0EBF
:1017C000046E00C300F0A5EC04F008C000F0005067
:0E17D0000F1302D000C30FF30FC300F012007E
:1017DE00220E0C6E086A096A0A6A0B6A0C06D8B4E5
:1017EE001FD0D8900B320A3209320832033202323D
:1017FE0001320032D8A0F2D70C06D8B409D004506A
:10180E0008260550092206500A2207500B22EAD755
:10181E00045008260550092206500A2207500B22B2
:02182E001200A6
:101830000450000A12E10550000A0FE10650000AA8
:101840000CE10750000A09E1FF0E006EFF0E016E69
:10185000FF0E026E7F0E036E99D00C6A07BE0C2A33
:101860000D6A0B6A0A6A096A086A035002100110BD
:101870000010D8B485D0035007180E6E0EBE0D1E92
:1018800007AE0BD0041E051E061E071E042AD8B480
:10189000052AD8B4062AD8B4072A03AE0BD0001EF6
:1018A000011E021E031E002AD8B4012AD8B4022A3F
:1018B000D8B4032A035007100E6E0EBE1DD029ECBB
:1018C00003F00CBE36D00DAE5BD0001E011E021E12
:1018D000031E002AD8B4012AD8B4022AD8B4032A95
:1018E000081E091E0A1E0B1E082AD8B4092AD8B4DD
:1018F0000A2AD8B40B2A44D007AE15D003BE0DD0A7
:1019000003500B6E02500A6E0150096E0050086EB3
:10191000036A026A016A006AD6D7036A026A016A28
:10192000006A002A000C031E021E011E001E0C8EFF
:10193000C6D7082AD8B4092AD8B40A2AD8B40B2A98
:101940000450085CD8A4BFD70550095CD8A4BBD705
:1019500006500A5CD8A4B7D707500B5CD8A4B3D7FD
:101960000B6A0A6A096A086A002AD8B4012AD8B43C
:10197000022AD8B4032A03AEA6D70E6A0E88FF0C3B
:0E1980000E6A0CA002D06DEC06F0000F1200F3
:10198E000FC302F010C303F002C000F003C001F059
:10199E00024A032A00C0E9FF01C0EAFFEE5201E04D
:1019AE00F3D703010F51025C006E10510358016E04
:0A19BE00010E005E000E015A120037
:1019C80013C300F003011307005228E00FC3E9FF17
:1019D80010C3EAFFEE50000A0CE00FC3E9FF10C382
:1019E800EAFF11C3D9FF12C3DAFFEE50DE1801E196
:1019F8000FD00FC3E9FF10C3EAFF11C3D9FF12C309
:101A0800DAFFDE50EE5C006E016A000E015A08D063
:101A180003010F4B102B114B122BD2D7006A016A0E
:021A28001200AA
:101A2A0003011D6B4DEC06F0800E0010096F0A6B66
:101A3A00000E0A13000E0A6F03011D6B09C21EF382
:0C1A4A0055EC04F00201236B246B120029
:101A56000301006B050E005D0AE200511125E16EDF
:101A6600000E1221E26E200EE66E002BF3D7005117
:101A76001125E16E000E1221E26EE66A00070051A2
:101A86001125136F000E1221146F0A0E046E000E3C
:101A9600056E0FC300F010C301F079EC06F008C024
:101AA60000F009C001F0300E002613C3E1FF14C395
:101AB600E2FF00C0E6FF0A0E046E000E056E0FC3BD
:101AC60000F010C301F079EC06F000C00FF301C07E
:101AD60010F3000E011802E1000E001801E102D019
:061AE6000007CDD712003D
:101AEC000301156B166B000E165D02E10A0E155DF7
:101AFC000BE215511325E16E16511421E26E200EE6
:101B0C00E66E154B162BEFD715511325E16E1651BA
:101B1C001421E26EE66A010E155F000E165B15517C
:101B2C001325176F16511421186F0A0E046E000E30
:101B3C00056E066E076E0FC300F010C301F011C3E3
:101B4C0002F012C303F0B4EC04F008C000F009C0BA
:101B5C0001F00AC002F00BC003F0300E002617C3D0
:101B6C00E1FF18C3E2FF00C0E6FF0A0E046E000E90
:101B7C00056E066E076E0FC300F010C301F011C3A3
:101B8C0002F012C303F0B4EC04F000C00FF301C078
:101B9C0010F302C011F303C012F3000E046E03180D
:101BAC0008E10450021805E10450011802E100504C
:101BBC00000A01E105D0010E155F000E165BAFD7D0
:021BCC00120005
:101BCE0002012351241101E017D003011D6B4DECCE
:101BDE0006F07F0E0014096F0A6B000E0A17000E36
:101BEE000A6F03011D6B09C21EF355EC04F0010EC2
:0A1BFE000201236F000E246F120095
:101C080000C008F00150006E016A026A036A0B6A9C
:101C18000C6A016A026A036A960E036E0A6A00AECB
:101C28001CEF0EF0081E001E082AD8B4002A0A8EDF
:101C380000C001F008C000F0086A026AB5EC08F0BC
:021C4800120088
:101C4A000B6A0350D8B46BEF0EF002500A6E028E84
:101C5A008E0E035E03AE6FEF0EF0036C080E035C8C
:101C6A00D8A04AEF0EF0036E013602C001F0026AF4
:101C7A00080E035CD8A04AEF0EF0036E0136016A23
:101C8A000350D8A4D89054EF0EF00350D8B454EFB0
:101C9A000EF0D89002320132032E4EEF0EF00BBC3A
:101CAA0001A061EF0EF0D8A061EF0EF0012AD8B4BE
:101CBA00022A02BE7EEF0EF00AAE84EF0EF0021E7A
:101CCA00011E012AD8B4022A84EF0EF0026A016AC0
:101CDA0084EF0EF00B800BAE88EF0EF0026A0AAEAC
:101CEA0088EF0EF0FF0E026E016E0A36023288EF9E
:101CFA000EF0010E0C6E94EC06F08AEF0EF0000E58
:101D0A000C6E8AEF0EF0FF0E0C6E0150006E025040
:041D1A00016E120044
:101D1E000D0E03012E6F0EEC00F00A0E03012E6F56
:061D2E000EEC00F01200B3
:101D34000301006B080E005D0BE20051010F1D6FE3
:101D44001E6B1F6B206B216B2AEC06F0002BF2D765
:021D540012007B
:101D5600030E006E0FC316F3000E0301176F00503B
:101D660005E0163716911737FF0FFAD7006BA00E4E
:101D76000F25F66E4A0EF76E000EF722000EF86E6D
:101D8600000EF8220900F5CF72F1146B156B000EE8
:101D9600155D02E1080E145DD8B09AD0200E126FC0
:101DA600000E136F000E006E1351005C02E112511B
:101DB600000819E2720E1225E16E010E1321E26E81
:101DC600010E125D006E000E1359016E720E002494
:101DD600E96E010E0120EA6EEECFE6FF010E125FFC
:101DE600000E135BDFD716511425006E175115210F
:101DF600016EA00E0024F66E4A0E0120F76E000E4C
:101E0600F86E000EF8220900F5CF72F1006B080E8D
:101E1600126F000E136F000E006E1351005C02E18C
:101E2600125100083EE212C31DF3720EE96E010E56
:101E3600EA6E0051E926D8B0EA2AEECF1EF3080E64
:101E46000025006E016A000E0122720E0024E96E62
:101E5600010E0120EA6EEECF1FF3100E0025006E74
:101E6600016A000E0122720E0024E96E010E0120A5
:101E7600EA6EEECF20F3180E0025006E016A000E02
:101E86000122720E0024E96E010E0120EA6EEECFE9
:101E960021F32AEC06F0002B010E125F000E135BF5
:101EA600BAD7126B136B1151135D02E11051125D1B
:101EB6000CE2060E0C6E300E0D6E0D2EFED70C2E9D
:101EC600FCD70000124B132BEED7144B152B5FD704
:021ED6001200F8
:101ED800A69C10C3AAFF0FC3A9FFA69EA680A8CFE1
:041EE80000F01200F4
:101EEC003E0E03011D6F4DEC06F00050200A01E17F
:101EFC0044D067DE020E03011D6F4DEC06F0BF0EE1
:101F0C00001403011E6F020E1D6F55EC04F003014B
:101F1C001D6B1E6B55EC04F0010E03011D6F590E69
:101F2C001E6F55EC04F0020E03011D6F230E1E6F85
:101F3C0055EC04F0030E03011D6F070E1E6F55ECDC
:101F4C0004F0040E03011D6F280E1E6F55EC04F0F7
:101F5C00050E03011D6F120E1E6F55EC04F0060EDC
:101F6C0003011D6F160E1E6F55EC04F03E0E03019F
:0C1F7C001D6F200E1E6F55EC04F01200CB
:101F8800F7C204F0F8C205F0F5C202F0F6C203F099
:101F9800F9C200F0FAC201F0010E0201F95F000E69
:101FA800FA5B005001100FE004C0E9FF05C0EAFF2A
:101FB80002C0E1FF03C0E2FFEECFE6FF024A032AB8
:101FC800044A052AE5D7F5C200F0F6C201F012006E
:101FD800F7C2F6FFF8C2F7FFF9C2F8FF0900F5CF1C
:101FE80000F0005218E0F7C2F6FFF8C2F7FFF9C296
:101FF800F8FF0900F5CF00F0F5C2E1FFF6C2E2FFF5
:1020080000C0E6FF0201F54BF62B010EF727000E84
:10201800F823F923DDD7F5C2E1FFF6C2E2FFE66A4D
:022028001200A4
:10202A00360E0101FC6F000EFD6F000EFE6F000EF2
:10203A00FF6F9E0E0201016F000E026F000E036F0A
:10204A00000E046F560E0101F06F020EF16F000EC2
:10205A00F26F000EF36FE60ECE6F020ECF6F220EF6
:10206A00D06F030ED16FAE0ED26F030ED36F220E56
:10207A00D46F030ED56FAA0ED66F030ED76F000E5C
:10208A00D86F000ED96F959295908C928C9095820C
:0C209A0095806D9E6D9C380E6C6E1200DF
:1020A6003F0E806E0F01386B388138831F0E926E9B
:1020B600929A899A546BFF0E816E830E936E396BDA
:1020C600826A3A6BFF0E946E948E949C94908B80E9
:1020D600836A3B6BFF0E956E95909482959C948EC9
:0420E600606A12001A
:1020EA001C0E0101E86F000EE96F2E0EEA6F030E57
:1020FA00EB6F8C0EEC6F000EED6F000EEE6F000EA4
:10210A00EF6F820EE46F000EE56F000EE66F000EB1
:10211A00E76FDA0EDA6F010EDB6F000EDC6F000E6E
:10212A00DD6FAC8A900EAB6E948E949C9EAA03D0FF
:08213A00AECF00F0FBD712004C
:102142000900F5CFE6FF0006FBE10106F9E1120006
:10215200F5C2E9FFF6C2EAFFEE5000080FE2F5C24F
:10216200E9FFF6C2EAFFEECF0FF3F7C210F3F8C2AF
:0E21720011F3F0DD0201F54BF62BEAD7120057
:102180000201F551070803E2006A016A28D0F5C28E
:1021900000F000360090003600900050C2121A0E77
:1021A0000C6EF80E0D6E0D2EFED70C2EFCD7000017
:1021B000C28200000000C2A201D0FDD700000000D2
:1021C000C3CF03F0000E046EC4CF01F0006A0350C9
:1021D00000260450012200C003F001C004F01200E8
:1021E0000050086E0150006E016A026A036A0B6AB1
:1021F0000C6A960E036E0A6A00C001F008C000F077
:0A220000086A026AB5EC08F012004B
:10220A00F5C204F0F6C205F004C0E9FF05C0EAFF12
:10221A00EE5203E0044A052AF7D704C002F005C0CB
:10222A0003F0044A052AF7C200F0F8C201F00201DD
:10223A00F74BF82B00C0E9FF01C0EAFF02C0E1FF3B
:10224A0003C0E2FFEECFE6FF02C0E9FF03C0EAFFE8
:10225A00EE5201E0E2D7F5C200F0F6C201F0120038
:10226A000201FD6BFE6BF5C201F3F6C202F3F7C27F
:10227A0003F3F8C204F3800EF819006E800E005CB6
:10228A0008E1000EF75D05E1000EF65D02E1000EC1
:10229A00F55D19E2010EFD6F000EFE6F0301016B81
:1022AA00026B036B046B0201F5510301015F02012A
:1022BA00F6510301025B0201F7510301035B0201BC
:1022CA00F8510301045B01C30FF302C310F303C304
:1022DA0011F304C312F3F9C213F3FAC214F301DCC3
:1022EA000B0E0201FB6F000EFC6F000E006EFC511C
:1022FA00005C02E1FB51000819E2FB51F925E16E8D
:10230A00FC51FA21E26E010EFB5D006E000EFC59D3
:10231A00016E0050F925E96E0150FA21EA6EEECFFE
:10232A00E6FF010EFB5F000EFC5BDFD7F9C2E1FF9F
:10233A00FAC2E2FF200EE66EFD51FE111AE0FB6BB7
:10234A00FC6BFB51F925E96EFC51FA21EA6EEE505D
:10235A00200A03E1FB4BFC2BF4D7010EFB5F000EB6
:10236A00FC5BFB51F925E16EFC51FA21E26E2D0E60
:04237A00E66E1200F9
:10237E000201F76BF86BF5C203F0F6C204F0F5C27A
:10238E0005F0F6C206F003C0E9FF04C0EAFFEE5006
:10239E00200A04E1F751F81101E110D0010EF76F98
:1023AE00000EF86F03C0E9FF04C0EAFF05C0E1FFAD
:1023BE0006C0E2FFEECFE6FF054A062A03C001F093
:1023CE0004C002F0034A042A01C0E9FF02C0EAFF7A
:1023DE00EE50000AD8E1F5C200F0F6C201F012008C
:1023EE00F6C200F00032009E0032009E0032009EC7
:1023FE000032009EF40E0024F66E530EF76E000EA1
:10240E00F722000EF86E000EF8220900F5CF00F04C
:10241E00F7C2E1FFF8C2E2FF00C0E6FF010E0201C3
:10242E00F725E16E000EF821E26E0F0EF615006E26
:10243E00F40E0024F66E530EF76E000EF722000E09
:10244E00F86E000EF8220900F5CF00F000C0E6FF8E
:10245E00020EF725E16E000EF821E26EF5C200F0D5
:10246E000032009E0032009E0032009E0032009E1E
:10247E00F40E0024F66E530EF76E000EF722000EC9
:10248E00F86E000EF8220900F5CF00F000C0E6FF4E
:10249E00030EF725E16E000EF821E26E0F0EF51514
:1024AE00006EF40E0024F66E530EF76E000EF72239
:1024BE00000EF86E000EF8220900F5CF00F000C0F5
:1024CE00E6FF040EF725E16E000EF821E26EE66AD5
:0224DE001200EA
:1024E0000201F96BFA6BF751F92503010F6F020135
:1024F000F851FA210301106FEFDC00C0FBF2000E6F
:102500000201FC6F000EFC1902E1000EFB1901E153
:1025100023D0800E006E800EFA19005C02E1F951A2
:102520003F0801E219D0F951F525E16EFA51F62183
:10253000E26EFBC2E6FF060E0C6E300E0D6E0D2E27
:10254000FED70C2EFCD70000F94BFA2B000EFC191D
:1025500002E1000EFB19C7E1F951F525006EFA51B1
:10256000F621016E010E005CE16E000E0158E26E74
:04257000E66A120005
:102574000201F76BF86B8FEC0EF0310E03010F6F55
:10258400020E106FC7EC0CF000C0F5F201C0F6F2B9
:1025940000C00FF301C010F3B10E116F020E126FE1
:1025A4002BEC0DF0B10E0F6F020E106F1FEC09F043
:1025B4008FEC0EF002013151550AD8A4CED044510B
:1025C400230AD8A4CAD0800EF619006E800E005CCF
:1025D40002E1140EF55DD8A0C0D0510E03010F6FB7
:1025E400530E106F000E116F01EC09F0310E030150
:1025F4000F6F020E106F1FEC09F08FEC0EF0020E3D
:102604000201F96F000EFA6F800EFA19006E800E47
:10261400F619005C02E1F551F95D33E2310EF9255A
:10262400E96E020EFA21EA6EEECF01F001503B0A88
:1026340025E1310EF925E16E020EFA21E26EE66A19
:10264400240EF725FB6F020EF821FC6F310EF925DD
:1026540003010F6F020E0201FA210301106F020E33
:102664000F5F000E105B37EC0AF0FBC2E1FFFCC207
:10267400E2FF00C0E6FF0201F74BF82BF94BFA2BFF
:10268400C3D7446B240EF725E16E020EF821E26EE7
:10269400300E425D006E0A0E0002F3CF00F043518B
:1026A4000026300E005E00C0E6FF24C200F3C8EC32
:1026B4000BF000C02DF225C200F3C8EC0BF000C0F3
:1026C40019F226C200F3C8EC0BF000C02EF227C2A8
:1026D40000F3C8EC0BF000C000F228C200F3C8EC11
:1026E4000BF000C0CBF029C200F3C8EC0BF000C023
:1026F400CCF00001CD6B8FEC0EF00001CD6B8FECB4
:102704000EF015EC0DF0CDC00FF3000E0301106FA9
:10271400CCC011F3000E126FCBC013F3000E146F74
:1027240000C215F3000E166F2DC217F3000E186FBA
:1027340019C219F3000E1A6F2EC21BF3000E1C6F80
:10274400A1EC0AF0E20E03010F6F530E106F000E9E
:0C275400116F01EC09F0E7EC0DF0120031
:102760000201FB51000805E3070EFC6F000EFD6F30
:1027700012D0FB51160805E2170EFE6F000EFF6F18
:1027800006D0FB51010FFE6FFF6B000EFF23FEC250
:10279000FCF2FFC2FDF2FCC207F3FDC208F3030125
:1027A000016B026B046A056A066A076AF5C200F0EB
:1027B000F6C201F0F7C202F0F8C203F03DEC09F0F6
:1027C000010ED8B0000E006E00520AE0F9C2E1FF1F
:1027D000FAC2E2FF2D0EE66E0201F94BFA2BF77FEB
:1027E000F5C204F0F6C205F0F7C206F0F8C207F031
:1027F000006A016A026A036A3DEC09F0010ED8B072
:10280000000E006E005238E0000E046E000E056EE1
:10281000000E066E7F0E076EF5C200F0F6C201F0E4
:10282000F7C202F0F8C203F03DEC09F0010ED8B097
:10283000000E006E005220E0F5C200F0F6C201F07A
:10284000F7C202F0F8C203F0000E046E000E056E2F
:10285000200E066E820E076EA4EC09F000C0F5F2A1
:1028600001C0F6F202C0F7F203C0F8F2010E030154
:10287000015F000E025BC8D7000E046E000E056EED
:10288000200E066E820E076EF5C200F0F6C201F051
:10289000F7C202F0F8C203F03DEC09F0000ED8B028
:1028A000010E006E00521EE0000E046E000E056E5A
:1028B000200E066E820E076EF5C200F0F6C201F021
:1028C000F7C202F0F8C203F0EDEC0AF000C0F5F236
:1028D00001C0F6F202C0F7F203C0F8F20301014BA7
:1028E000022BCAD703010151072702510823010E09
:1028F000036F000E046F000E096F000E0A6F000ECA
:102900000B6F7F0E0C6F800E0419006E800E08197D
:10291000005C02E10751035D1EE2000E046E000E32
:10292000056E200E066E820E076E09C300F00AC304
:1029300001F00BC302F00CC303F0EDEC0AF000C091
:1029400009F301C00AF302C00BF303C00CF3030147
:10295000034B042BD8D7000E046E000E056E000E3C
:10296000066E800E076E09C300F00AC301F00BC3A8
:1029700002F00CC303F0EDEC0AF0F5C204F0F6C26D
:1029800005F0F7C206F0F8C207F0A2EC06F000C0AE
:10299000F5F201C0F6F202C0F7F203C0F8F2000E41
:1029A000046E000E056E200E066E820E076E3DEC64
:1029B00009F0000ED8B0010E006E00520CE0000EBF
:1029C0000201F56F000EF66F000EF76F7F0EF86FC5
:1029D0000301014B022B0301800E0219006E800ED1
:1029E000005C02E1000E015D3CE2F9C2E1FFFAC2C7
:1029F000E2FF300EE66E0201F94BFA2BF9C2E1FF5D
:102A0000FAC2E2FF2E0EE66EF94BFA2B800E03019E
:102A10000819006E800E005C02E1000E075D04E202
:102A20000751015F0851025BFF0E036FFF0E046F39
:102A3000800E0219006E800E0419005C02E1035141
:102A4000015D0FE2F9C2E1FFFAC2E2FF300EE66E6D
:102A50000201F94BFA2B010E0301035F000E045B28
:102A6000E7D7036B046B800E0419006E800E081903
:102A7000005C02E10751035D67E2F5C200F0F6C2B7
:102A800001F0F7C202F0F8C203F025EC0EF000C02E
:102A900005F301C006F3300E0026F9C2E1FFFAC2C9
:102AA000E2FF00C0E6FF0201F94BFA2B03010451DB
:102AB000021902E10151031909E1F9C2E1FFFAC269
:102AC000E2FF2E0EE66E0201F94BFA2B05C300F071
:102AD00006C301F004EC0EF000C009F301C00AF3D4
:102AE00002C00BF303C00CF300C004F001C005F0FA
:102AF00002C006F003C007F0F5C200F0F6C201F014
:102B0000F7C202F0F8C203F03AEC09F000C0F5F2A7
:102B100001C0F6F202C0F7F203C0F8F2000E046E34
:102B2000000E056E200E066E820E076EA4EC09F0F4
:102B300000C0F5F201C0F6F202C0F7F203C0F8F2ED
:102B40000301034B042B8FD7F9C2E1FFFAC2E2FF66
:042B5000E66A12001F
:102B54000201F86B030EF85D0AE2F851F625E16E06
:102B6400000EF721E26E200EE66EF82BF3D7F85133
:102B7400F625E16E000EF721E26EE66AF807F851D9
:102B8400F625F96F000EF721FA6F0A0E046EF5C2EE
:102B940000F0A5EC04F008C000F0300E0026F9C2E5
:102BA400E1FFFAC2E2FF00C0E6FF0A0E046EF5C2BE
:102BB40000F0A5EC04F000C0F5F20050000A01E1B9
:082BC40002D0F807DCD7120073
:102BCC00000E0201F61902E1000EF5193AE0F5C209
:102BDC00E9FFF6C2EAFFEE5234E0F7C20FF3F8C297
:102BEC0010F3C7EC0CF000C013F3F5C20FF3F6C2F0
:102BFC0010F3F7C211F3F8C212F3E4EC0CF0000E70
:102C0C00011802E1000E001805E1F5C200F0F6C251
:102C1C0001F019D0010E0201F52503010F6F000E12
:102C2C000201F6210301106FF7C2E9FFF8C2EAFFB7
:102C3C00EECF11F3AAEC0BF000C0F5F201C0F6F2E6
:082C4C00BFD7006A016A120003
:102C5400060E0201F525E96E000EF621EA6EC00E9D
:102C6400EE24F76F120EEE20F86F000EF96FFA6F74
:102C7400F7C200F0F8C201F0F9C202F0FAC203F0A0
:102C84000C0E046E000E056E066E076EEFEC0BF074
:102C940000C0F7F201C0F8F202C0F9F203C0FAF280
:102CA400050EF525E96E000EF621EA6E030EEE5CC4
:102CB400046E056A000E055A045000240301096FCE
:102CC400055001200A6F000E05BEFF0E02200B6F97
:102CD400000E05BEFF0E03200C6F09C3F7F20AC3F2
:102CE400F8F20BC3F9F20CC3FAF20C0E046E000EE8
:102CF400056E066E076E09C300F00AC301F00BC32C
:102D040002F00CC303F018EC0CF008C000F009C08A
:102D140001F00AC002F00BC003F000C004F001C0CF
:102D240005F002C006F003C007F00436049005362F
:102D340006360736070E04240301056F000E05202E
:102D4400066F000E0620076F000E0720086F6D0E39
:102D5400006E010E016E000E026E036E09C304F0D4
:102D64000AC305F00BC306F00CC307F0EFEC0BF03D
:102D7400055100260651012207510222085103225F
:102D84000C0E046E000E056E066E076E18EC0CF049
:102D940000C005F301C006F302C007F303C008F343
:102DA40005C3FBF206C3FCF207C3FDF208C3FEF23F
:102DB400030E0201F525E96E000EF621EA6E300ECF
:102DC400046E000E056E066E076E09C300F00AC39A
:102DD40001F00BC302F00CC303F018EC0CF0EE503E
:102DE4000026000E012202220322530E005E7D0EF5
:102DF400015A000E025A035A005003010525046EBD
:102E040001500621056E02500721066E0350082169
:102E1400076E04C0FBF205C0FCF206C0FDF207C059
:102E2400FEF2800E000A006E800E0718005C08E1B6
:102E34000650230805E10550150802E10450230853
:102E44004FE2C00E046E120E056E000E066E076E83
:102E5400F7C200F0F8C201F0F9C202F0FAC203F0BE
:102E640018EC0CF000C005F301C006F302C007F330
:102E740003C008F3B00E046E040E056E000E066E59
:102E8400076EF7C200F0F8C201F0F9C202F0FAC20C
:102E940003F018EC0CF005C304F006C305F007C3F7
:102EA40006F008C307F00050045E0150055A0250B2
:102EB400065A0350075A260E0424006E000E0520FD
:102EC400016E000E0620026E000E0720036E0050F5
:102ED4000201FB270150FC230250FD230350FE2373
:102EE4000201040EF5250301056F000E0201F6210F
:102EF4000301066F070E046E000E056E066E076E64
:102F0400FBC200F0FCC201F0FDC202F0FEC203F0FD
:102F140018EC0CF008C000F009C001F00AC002F07F
:102F24000BC003F005C3E1FF06C3E2FF00C0E6FFE8
:102F3400020E0201F525E96E000EF621EA6EEECFCF
:102F440001F3000E0301026F036F046F000E026FA2
:102F5400036F046F01C300F002C301F003C302F066
:102F640004C303F0100E046E0E0E056E000E066E02
:102F7400076EEFEC0BF000C001F301C002F302C0D6
:102F840003F303C004F3010E0201F525E96E000EFC
:102F9400F621EA6EEECF04F03C0E0402F3CF04F007
:102FA400F4CF05F0000E05BEFF0E066E076E00504E
:102FB400042601500522025006220350072204C0B1
:102FC40001F305C002F306C003F307C004F3F5C21E
:102FD400E9FFF6C2EAFFEECF00F00050042403013B
:102FE400056F000E0520066F000E0620076F000E09
:102FF4000720086F05C301F306C302F307C303F3F5
:1030040008C304F3FBC200F0FCC201F0FDC202F0ED
:10301400FEC203F05850005E5950015A5A50025AE9
:103024005B50035A800E046E510E056E010E066E3F
:10303400000E076EEFEC0BF005510026065101223D
:0A3044000751022208510322120076
:10304E000F01429F428B4299C280C19EC196C1948C
:10305E00C192C180C08EC08AC088C096C082C09402
:04306E00C0901200FC
:0E3072009488949A94968298829A829612007C
:103080004FEC00F0D00E0301226FD7EC01F00301EA
:10309000226BD7EC01F02BEC01F0D10E0301226F73
:1030A000D7EC01F0010E0301226F73EC01F001C3B4
:1030B000E1FF02C3E2FF00C0E6FF010E0301226F41
:1030C00073EC01F003C3E1FF04C3E2FF00C0E6FFBD
:1030D000010E0301226F73EC01F005C3E1FF06C38B
:1030E000E2FF00C0E6FF010E0301226F73EC01F066
:1030F00007C3E1FF08C3E2FF00C0E6FF010E0301C2
:10310000226F73EC01F009C3E1FF0AC3E2FF00C0C4
:10311000E6FF010E0301226F73EC01F00BC3E1FF28
:103120000CC3E2FF00C0E6FF0301226B73EC01F069
:103130000DC3E1FF0EC3E2FF00C0E6FFD5EC01F0D6
:0231400012007B
:1031420001C3E9FF02C3EAFFEECF03F0700E0314DE
:10315200026E02C000F00032009E0032009E003279
:10316200009E0032009E0A0E0002F3CF01F00F0E05
:103172000314006E01C3E1FF02C3E2FF0050012409
:10318200E66E03C3E9FF04C3EAFFEECF03F0F00EDD
:103192000314026E02C000F00032009E0032009E54
:1031A2000032009E0032009E0A0E0002F3CF01F0B0
:1031B2000F0E0314006E03C3E1FF04C3E2FF0050CD
:1031C2000124E66E05C3E9FF06C3EAFFEECF03F072
:1031D200300E0314026E02C000F00032009E003274
:1031E200009E0032009E0032009E0A0E0002F3CFC3
:1031F20001F00F0E0314006E05C3E1FF06C3E2FFE8
:1032020000500124E66E07C3E9FF08C3EAFF07C3C3
:10321200E1FF08C3E2FF070EEE1609C3E9FF0AC386
:10322200EAFFEECF03F0F00E0314026E02C000F0CC
:103232000032009E0032009E0032009E0032009E4C
:103242000A0E0002F3CF01F00F0E0314006E09C341
:10325200E1FF0AC3E2FF00500124E66E0BC3E9FF5F
:103262000CC3EAFFEECF03F0100E0314026E02C08D
:1032720000F00032009E0032009E0032009E0032BA
:10328200009E0A0E0002F3CF01F00F0E0314006E2F
:103292000BC3E1FF0CC3E2FF00500124E66E0DC335
:1032A200E9FF0EC3EAFFEECF03F0F00E0314026E45
:1032B20002C000F00032009E0032009E0032009EEA
:1032C2000032009E0A0E0002F3CF01F00F0E03142B
:1032D200006E0DC3E1FF0EC3E2FF00500124E66E53
:0232E2001200D8
:1032E4000A0E046EF9C200F0A5EC04F0300E0024BE
:1032F40002010B6F0A0E046EF9C200F0A5EC04F093
:1033040008C000F0300E00240C6F2F0E0D6F0A0E53
:10331400046E19C200F0A5EC04F0300E00240E6F08
:103324000A0E046E19C200F0A5EC04F008C000F007
:10333400300E00240F6F2F0E106F320E116F300EEF
:10334400126F0A0E046EFBC200F0A5EC04F0300EFE
:103354000024136F0A0E046EFBC200F0A5EC04F007
:1033640008C000F0300E0024146F156B0A0E046EB2
:10337400F7C200F0A5EC04F0300E00241A6F0A0E18
:10338400046EF7C200F0A5EC04F008C000F0300EA3
:1033940000241B6F3A0E1C6F0A0E046EF6C200F076
:1033A400A5EC04F0300E00241D6F0A0E046EF6C264
:1033B40000F0A5EC04F008C000F0300E00241E6FED
:1033C4003A0E1F6F0A0E046EF5C200F0A5EC04F06D
:1033D400300E0024206F0A0E046EF5C200F0A5EC36
:1033E40004F008C000F0300E0024216F226B12009C
:1033F400F5C2F6FFF6C2F7FFF7C2F8FF0900F5CFF2
:1034040001F00150000816E2F5C2F6FFF6C2F7FF1C
:10341400F7C2F8FF0900F5CF0FF3F8C210F3F9C2B1
:1034240011F3ABEC0EF0010E0201F527000EF623AA
:06343400F723DED71200B1
:10343A000001C96BCA6B000ECA5D02E1800EC95D4C
:10344A0012E2310EC925E16E020ECA21E26EE66A67
:10345A00010EC925006E000ECA21016E00C0C9F016
:10346A0001C0CAF0E8D7C96BCA6BC46BC56BAECFD3
:0C347A00C6F0C66BC76BC86B9D8A1200C1
:10348600F5C204F0F6C205F004C002F005C003F070
:10349600044A052AF7C200F0F8C201F00201F74B10
:1034A600F82B00C0E9FF01C0EAFF02C0E1FF03C03C
:1034B600E2FFEECFE6FF02C0E9FF03C0EAFFEE52ED
:0E34C60001E0E2D7F5C200F0F6C201F01200FC
:1034D4008B80090E03011D6F1E6B1F6B206B216B0C
:1034E4002AEC06F00A0E1D6F1E6B1F6B206B216BFE
:1034F4002AEC06F00B0E1D6F070E1E6F070E1F6FD2
:10350400070E206F070E216F2AEC06F00C0E1D6FBC
:10351400010E1E6F010E1F6F010E206F010E216F31
:103524002AEC06F00F0E1D6F1E6B1F6B206B216BB8
:103534002AEC06F0340E0C6EF10E0D6E0D2EFED735
:103544000C2EFCD7000000009AEC0EF0030E0B6E5C
:10355400080E0C6E770E0D6E0D2EFED70C2EFCD7BA
:063564000B2EFAD7120045
:10356A00CD6ACD9ECD9CCD82CD8ACD880B0ECF6EF5
:10357A00DC0ECE6E9E909F900201176B186B2F6B1C
:08358A00306BCD909D90120002
:103592009E900B0ECF6EDC0ECE6E0201176B186B77
:0A35A2002F6B306BCD809D8012006E
:1035AC0000C01AF001C019F0E1CF1BF0E2CF1CF003
:1035BC009DAA69D09EAA67D0AECFC6F0ABA20FD0A1
:1035CC00AB98AECFC6F0AB88010E0101DE25006EC4
:1035DC00000EDF21016E00C0DEF101C0DFF1ABA4F3
:1035EC000FD00101AB9EAB8E010EDE25006E000EDE
:1035FC00DF21016E00C0DEF101C0DFF1AECFC6F0FD
:10360C000001C6510D0A09E0000E006ECA51005CA3
:10361C0002E1C9517E0801E314D0010EC76F000E00
:10362C00C86F9D9A310EC925E16E020ECA21E26E59
:10363C00E66AC9C0C4F0CAC0C5F0C96BCA6BC66B18
:10364C0022D0000E006ECA51005C02E1C9517E0806
:10365C0004E2020EC76F000EC86F310EC925E16E71
:10366C00020ECA21E26EC6C0E6FFC9C0C4F0CAC0D1
:10367C00C5F0010EC925006E000ECA21016E00C0F6
:10368C00C9F001C0CAF0F2AA0CD0F2A40AD02A0EDA
:10369C00AD6E010E0101E027000EE123E223E323CE
:1036AC00F2941AC000F019C001F01BC0E1FF1CC05D
:0436BC00E2FF110018
:1036C00000C018F0156ED8CF16F0E0CF17F09DA00F
:1036D0001DD09EA01BD00201174B182B0101C35116
:1036E0000201185D04E10101C2510201175D09E305
:1036F0009D90176B186B010E2F6F000E306FCD90E1
:103700009D900B0ECF6EDB0ECE6E9E901750E06E2E
:0E3710001650D86E153A153818C000F010008B
:10371E0051EC2AF0720ED36E9B6A9B9CD26A150EE8
:10372E000B6E4B0E0C6EBE0E0D6E0D2EFED70C2EAE
:10373E00FCD70B2EFAD7000053EC10F08B80080E3E
:10374E000101C26F000EC36F899AB886B06ACF0EA0
:10375E00AF6EAC8475EC10F0030E0B6E080E0C6E93
:10376E00770E0D6E0D2EFED70C2EFCD70B2EFAD724
:10377E000C0E03012E6F0EEC00F00B0E0B6E260ED0
:10378E000C6E5D0E0D6E0D2EFED70C2EFCD70B2E75
:10379E00FAD700000000220E0101C46F010EC56FA2
:1037AE00D00E0001CE6F000ECF6F8FEC0EF0D00E4C
:1037BE0003010F6F530E106F000E116F01EC09F025
:1037CE000101206B216B000E215D02E1070E205DD1
:1037DE001CE2030E006E000E016E20C104F021C12A
:1037EE0005F07DEC04F0320E0024E96E000E01208F
:1037FE00EA6EEECF0FF3EECF10F3EECF11F301EC36
:10380E0009F00101204B212BDED7290E0B6E960EEF
:10381E000C6E7F0E0D6E0D2EFED70C2EFCD70B2EC2
:10382E00FAD78FEC0EF0800E0001A16F3E0EA26F44
:10383E00C4C1F5F2C5C1F6F2D10E0201F76F520EF8
:10384E00F86F000EF96FECEC0FF0A1C00FF3A2C0F1
:10385E0010F3B10E0301116F020E126F2BEC0DF06F
:10386E00170E0101C4250201F56F000E0101C521DD
:10387E000201F66FB10EF76F020EF86F050EF96FBB
:10388E00000EFA6FC4EC0FF0C4C10FF3C5C110F3F4
:10389E001FEC09F00201236B0A0E6E6E15EC10F090
:1038AE00AD0E03010F6F520E106F000E116F01EC73
:1038BE0009F076EC0FF0E7EC0DF00B0E0B6E260E0A
:1038CE000C6E5D0E0D6E0D2EFED70C2EFCD70B2E34
:1038DE00FAD700000000CD0E0301016F000E026F3B
:1038EE00CC0E036F000E046FCB0E056F000E066F2D
:1038FE00000E076F020E086F2D0E096F020E0A6F73
:10390E00190E0B6F020E0C6F2E0E0D6F020E0E6F38
:10391E0040EC18F0CD0E0301016F000E026FCC0EBD
:10392E00036F000E046FCB0E056F000E066F000EB8
:10393E00076F020E086F2D0E096F020E0A6F190E19
:10394E000B6F020E0C6F2E0E0D6F020E0E6FA1EC92
:10395E0018F0CDC0F5F2CCC0F6F2CBC0F7F200C233
:10396E00F8F22DC2F9F219C2FAF22EC2FBF2B3DC52
:10397E00040E03010F6F540E106F000E116F01EC49
:10398E0009F00B0E03010F6F020E106F1FEC09F002
:10399E00590E0F6F540E106F000E116F01EC09F0DF
:1039AE001A0E03010F6F020E106F1FEC09F08FEC51
:1039BE000EF0290E0B6E960E0C6E7F0E0D6E0D2EEA
:1039CE00FED70C2EFCD70B2EFAD70001A36B3B0EA5
:1039DE00A46F170EA56F1E0EA66F0C0EA86FE00E2D
:1039EE00A96F070EAA6FAB6BAC6BAD6B010EAE6F12
:1039FE00010EB06FE10EB16F070EB26F870E0301AD
:103A0E000F6F520E106F000E116F01EC09F0A30E26
:103A1E000201F56F000EF66F2AEC16F000C025F0CD
:103A2E0001C026F002C027F003C028F000C00FF33B
:103A3E0001C010F302C011F303C012F3B10E136FE5
:103A4E00020E146F76EC0DF0B10E0F6F020E106FAA
:103A5E001FEC09F08FEC0EF0150E03010F6F520ED6
:103A6E00106F000E116F01EC09F0AB0E0201F56F35
:103A7E00000EF66F2AEC16F000C01DF001C01EF00D
:103A8E0002C01FF003C020F000C00FF301C010F3FE
:103A9E0002C011F303C012F3B10E136F020E146FB6
:103AAE0076EC0DF0B10E0F6F020E106F1FEC09F0D9
:103ABE008FEC0EF0200E03010F6F540E106F000EE0
:103ACE00116F01EC09F0AB0E0201F56F000EF66FEF
:103ADE002AEC16F000C0F1F201C0F2F202C0F3F2CD
:103AEE0003C0F4F2A30E0201F56F000EF66F2AEC7E
:103AFE0016F0F1C204F0F2C205F0F3C206F0F4C201
:103B0E0007F00050045E0150055A0250065A035049
:103B1E00075A04C021F005C022F006C023F007C0EA
:103B2E0024F004C00FF305C010F306C011F307C054
:103B3E0012F3B10E136F020E146F76EC0DF0B10E80
:103B4E000F6F020E106F1FEC09F08FEC0EF09F90AE
:103B5E003B0E03010F6F520E106F000E116F01EC32
:103B6E0009F027EC18F0960E03010F6F500E106F30
:103B7E00000E116F01EC09F039EC18F0A4DC680EA0
:103B8E000F6F530E106F000E116F01EC09F09AECCF
:103B9E000EF0F28CD08EF28CF28EEB0E0F6F4F0E6B
:103BAE00106F000E116F01EC09F0080E0101C26FCB
:103BBE00000EC36FD3DCE6DC240EAD6E8FEC0EF080
:103BCE00000E0201301902E1000E2F1901E1F8D7A3
:103BDE00230EAD6E8FEC0EF0EB0E03010F6F510E38
:103BEE00106F000E116F01EC09F09AEC0EF07E0EC4
:103BFE000201F56F540EF66F000EF76F010EF86F9F
:103C0E00000EF96FFAEC19F0440E0201F56F540E26
:103C1E00F66F000EF76F050EF86F000EF96FFAECE7
:103C2E0019F0897A150E0B6E4B0E0C6EBE0E0D6EC4
:103C3E000D2EFED70C2EFCD70B2EFAD70000897A4C
:103C4E00220E0101C46F010EC56FC4C1F5F2C5C1CC
:103C5E00F6F26F0E0201F76F540EF86F000EF96F49
:103C6E00ECEC0FF000019F9B2F6A280E306E000EB9
:103C7E00316E1DEC1AF09AEC0EF0740E0201F56F17
:103C8E00540EF66F000EF76F010EF86F000EF96FFF
:103C9E00FAEC19F0220E0001CE6F010ECF6FCD0E91
:103CAE000301016F000E026FCC0E036F000E046F46
:103CBE00CB0E056F000E066F000E076F020E086F1B
:103CCE002D0E096F020E0A6F190E0B6F020E0C6F7E
:103CDE002E0E0D6F020E0E6F40EC18F0CD0E03017E
:103CEE00016F000E026FCC0E036F000E046FCB0E31
:103CFE00056F000E066F000E076F020E086F2D0E79
:103D0E00096F020E0A6F190E0B6F020E0C6F2E0E3C
:103D1E000D6F020E0E6FA1EC18F0CDC0F5F2CCC0F7
:103D2E00F6F2CBC0F7F200C2F8F22DC2F9F219C2C8
:103D3E00FAF22EC2FBF272EC19F03B0E0001AB6FE1
:103D4E003B0EAC6F170EAD6F1F0EAE6F0C0EB06F3D
:103D5E00E00EB16F070EB26FCDC0A3F0CCC0A4F0D1
:103D6E00CBC0A5F02DC2A6F019C2A8F0D00E006EE1
:103D7E00070E016E02012E510026D8B0012A00C096
:103D8E00A9F001C0AAF0D00E0001CE6F000ECF6FC9
:103D9E00CEC0F5F2CFC0F6F20B0E0201F76F020E97
:103DAE00F86F43EC1AF0CEC00FF3CFC010F3C7EC90
:103DBE000CF000C0C2F001C0C3F000500001CE25CF
:103DCE000201F56F01500001CF210201F66F2D0E99
:103DDE00F76F000EF86F05EC11F0CEC00FF3CFC0E9
:103DEE0010F3C7EC0CF000C0C2F001C0C3F00050DD
:103DFE000001CE250201F56F01500001CF21020115
:103E0E00F66F1A0EF76F020EF86F05EC11F0120E28
:103E1E0003010F6F540E106F000E116F01EC09F0BD
:103E2E00CEC00FF3CFC010F31FEC09F08D0E0F6F45
:103E3E00540E106F000E116F01EC09F0A30E02016B
:103E4E00F56F000EF66F2AEC16F000C025F001C0DB
:103E5E0026F002C027F003C028F000C00FF301C007
:103E6E0010F302C011F303C012F3B10E136F020E62
:103E7E00146F76EC0DF0B10E0F6F020E106F1FEC7B
:103E8E0009F08FEC0EF0610E03010F6F520E106FE2
:103E9E00000E116F01EC09F0AB0E0201F56F000E72
:103EAE00F66F2AEC16F000C01DF001C01EF002C025
:103EBE001FF003C020F000C0F5F201C0F6F202C000
:103ECE00F7F203C0F8F2B10E0201F96F020EFA6FAB
:103EDE0035EC11F0B10E03010F6F020E106F1FECD7
:103EEE0009F08FEC0EF0AB0E0201F56F000EF66FBF
:103EFE002AEC16F000C0F1F201C0F2F202C0F3F2A9
:103F0E0003C0F4F2A30E0201F56F000EF66F2AEC59
:103F1E0016F0F1C221F0F2C222F0F3C223F0F4C285
:103F2E0024F00050215E0150225A0250235A0350B1
:103F3E00245AF50E0F6F520E106F000E116F01EC1A
:103F4E0009F021C0F5F222C0F6F223C0F7F224C028
:103F5E00F8F2B30E0201F96F000EFA6F35EC11F0A4
:103F6E00B30EF56F000EF66FBFEC11F0B30E03013A
:103F7E000F6F000E106F1FEC09F08FEC0EF0800E1D
:103F8E002418006E800E005C08E1000E235C05E133
:103F9E00000E225C02E1040E215C41E27F0E006EF7
:103FAE00800E2418005C08E12350FF0805E1225022
:103FBE00FF0802E12150880832E2010E0101C26FB2
:103FCE00000EC36FCEC0F5F2CFC0F6F2940E020112
:103FDE00F76F510EF86F000EF96FECEC0FF0CEC0CC
:103FEE000FF3CFC010F31FEC09F08FEC0EF0C4C12D
:103FFE00F5F2C5C1F6F2830E0201F76F540EF86F9B
:10400E00000EF96FECEC0FF0CEC0F5F2CFC0F6F269
:10401E00140E0201F76F000EF86FA9EC10F0800E6F
:10402E00006E800E2418005C08E12350000805E1A4
:10403E002250000802E12150040848E2800E2418A4
:10404E00006E800E005C08E1000E235C05E1010E9F
:10405E00225C02E12C0E215C39E2020E0101C26FDC
:10406E00000EC36FD00E0001CE6F000ECF6FCEC00C
:10407E00F5F2CFC0F6F2880E0201F76F540EF86F0C
:10408E00000EF96FECEC0FF0CEC0F5F2CFC0F6F2E9
:10409E00B30E0201F76F000EF86F05EC11F0CEC0F3
:1040AE00F5F2CFC0F6F2290EF76F000EF86F05ECA1
:1040BE0011F0C4C1F5F2C5C1F6F29B0EF76F540EA6
:1040CE00F86F000EF96FECEC0FF049D00A0E0101FB
:1040DE00C26F000EC36FD00E0001CE6F000ECF6FF9
:1040EE00CEC0F5F2CFC0F6F20B0E0201F76F020E44
:1040FE00F86F43EC1AF0CEC00FF3CFC010F3C7EC3D
:10410E000CF000C0C2F001C0C3F000500001CE257B
:10411E000201F56F01500001CF210201F66F2B0E47
:10412E00F76F000EF86F05EC11F0CEC00FF3CFC095
:10413E0010F3C7EC0CF000C0C2F001C0C3F0005089
:10414E000001CE250201F56F01500001CF210201C1
:10415E00F66F1A0EF76F020EF86F05EC11F00001F4
:10416E009FABF7D0010E2F14016E0150010AD8A497
:10417E00F0D00A0E0101C26F000EC36F9AEC0EF062
:10418E00920E0201F56F540EF66F000EF76F010ED0
:10419E00F86F000EF96FFAEC19F0D00E0001CE6F29
:1041AE00000ECF6FCEC0F5F2CFC0F6F2970E020121
:1041BE00F76F540EF86F000EF96FECEC0FF0CEC0E7
:1041CE000FF3CFC010F3C7EC0CF000C0C2F001C06B
:1041DE00C3F00201F56BC0EC10F000C0F4F101C0A9
:1041EE00F5F1CEC00FF3CFC010F31FEC09F0F4C100
:1041FE000FF3F5C110F3B10E116F020E126F2BEC0F
:10420E000DF0B10E0F6F020E106F1FEC09F0680E5D
:10421E000F6F540E106F000E116F01EC09F0F4C108
:10422E0000F0F5C101F0F0EC10F0470E046E030E35
:10423E00056E780E066E7C0E076EA4EC09F0CD0EA0
:10424E00046ECC0E056EE00E066E830E076EA2ECAB
:10425E0006F000C0F6F101C0F7F102C0F8F103C09C
:10426E00F9F100C0F5F201C0F6F202C0F7F203C098
:10427E00F8F2B10E0201F96F020EFA6F010EFB6F2A
:10428E00B0EC13F00001C251CE250201F56F000112
:10429E00C351CF210201F66FB10EF76F020EF86F08
:1042AE0005EC11F0CEC00FF3CFC010F3C7EC0CF03D
:1042BE0000C0C2F001C0C3F000500001CE250201C3
:1042CE00F56F01500001CF210201F66F9E0EF76FC0
:1042DE00540EF86F000EF96FECEC0FF0CEC00FF32A
:1042EE00CFC010F31FEC09F08FEC0EF0CEC00FF321
:1042FE00CFC010F3C7EC0CF000C0C2F001C0C3F089
:10430E000101206B216B0001C3510101215D04E10C
:10431E000001C2510101205D1CE220510001CE2599
:10432E00E96E010121510001CF21EA6EEE50B00A73
:10433E000CE1010120510001CE25E16E0101215158
:10434E000001CF21E26E7E0EE66E0101204B212B85
:10435E00DAD7390E03010F6F540E106F000E116F66
:10436E0001EC09F02FC0F5F2B10E0201F66F020E4C
:10437E00F76FAAEC15F0B10E03010F6F020E106F5E
:10438E001FEC09F0090E2E6F0EEC00F0010E2F142B
:10439E00016E0150010A11E1CEC0F5F2CFC0F6F266
:1043AE00140E0201F76F000EF86FA9EC10F0310E2B
:1043BE0003012E6F0EEC00F010D0C4C1F5F2C5C192
:1043CE00F6F20A0E0201F76F000EF86FA9EC10F06C
:1043DE00300E03012E6F0EEC00F08FEC0EF02F2A34
:1043EE00B5EC1AF0C9EC1AF00201000E301902E118
:1043FE00000E2F1908E1000E0001C81902E1000E8F
:10440E00C71901E1F1D70001000EC81902E1010E32
:10441E00C719D8A43BD3310E0201F56F020EF66F09
:10442E00860EF76F000EF86FE6EC15F000C0FAF18D
:10443E0001C0FBF1000E026E0150025C02E1005061
:10444E00000843E2310E03010F6F020E106FC7EC2E
:10445E000CF0800E026E800E0118025C02E100501C
:10446E00060833E2310E0F6F020E106FC7EC0CF020
:10447E0000C0C2F001C0C3F0000E026E0150025C1B
:10448E0002E10050060821E2000E0001C35D02E1C8
:10449E00540EC25D1AE25C0E03010F6F000E106F18
:1044AE001FEC09F0350E0F6F020E106F1FEC09F0A6
:1044BE008FEC0EF0C4C1F5F2C5C1F6F2350E020155
:1044CE00F76F020EF86F43EC1AF00201310EF56F22
:1044DE00020EF66F750EF76F000EF86FE6EC15F024
:1044EE0000C0FAF101C0FBF1000E026E0150025C39
:1044FE0002E10050000815E200019F8B310E03010E
:10450E000F6F020E106FC7EC0CF000C0C2F001C0AE
:10451E00C3F0950E0F6F530E106F000E116F01EC5E
:10452E0009F0310E0201F56F020EF66F7D0EF76F78
:10453E00000EF86FE6EC15F000C0FAF101C0FBF1C9
:10454E00000E026E0150025C02E1005000080BE208
:10455E0000019F9B650E03010F6F510E106F000E31
:10456E00116F01EC09F0310E0201F56F020EF66FBC
:10457E00980EF76F000EF86FE6EC15F000C0FAF12A
:10458E0001C0FBF1000E026E0150025C02E1005010
:10459E000008D8B08DD0310E03010F6F020E106FD0
:1045AE00C7EC0CF000C0C2F001C0C3F0000E026EEA
:1045BE000150025C02E100500608D8B079D0020129
:1045CE00056B066B0101206B216B060E0001C25DAF
:1045DE00016E000EC359026E02500101215D02E10F
:1045EE000150205D1DE2370E2025E96E020E2121BD
:1045FE00EA6EEECF01F0300E015C0EE3370E202591
:10460E00E96E020E2121EA6EEECF01F0015039085B
:10461E0003E30201054B062B0101204B212BD5D7BD
:10462E00060E0001C25D016E000EC359026E02013C
:10463E000651021802E1015005193AE1370E030145
:10464E000F6F020E106F37EC0AF000C007F201C0B8
:10465E0008F2000E026E0150025C02E100500108E9
:10466E000BE2020E0201085D02E1000E075D04E29C
:10467E0007C230F008C231F0AB0E03010F6F530EBC
:10468E00106F000E116F01EC09F030C00FF331C046
:10469E0010F3B10E0301116F020E126F2BEC0DF021
:1046AE00B10E0F6F020E106F1FEC09F08FEC0EF0B3
:1046BE00310E0201F56F020EF66F900EF76F000EBF
:1046CE00F86FE6EC15F000C0FAF101C0FBF1000E38
:1046DE00026E0150025C02E100500008D8B0C5D055
:1046EE00310E03010F6F020E106FC7EC0CF000C0FD
:1046FE00C2F001C0C3F0000E026E0150025C02E176
:10470E0000500708D8B0B1D0000E0001C35D02E121
:10471E000A0EC25DD8B0A9D00201056B066B01016D
:10472E00206B216B070E0001C25D016E000EC35996
:10473E00026E02500101215D02E10150205D1DE279
:10474E00380E2025E96E020E2121EA6EEECF01F021
:10475E00300E015C0EE3380E2025E96E020E21218B
:10476E00EA6EEECF01F00150390803E30201054B6A
:10477E00062B0101204B212BD5D7070E0001C25D60
:10478E00016E000EC359026E02010651021802E1BB
:10479E00015005196AE1380E03010F6F020E106FFA
:1047AE0037EC0AF000C007F201C008F2610E0F6F7D
:1047BE00540E106F000E116F01EC09F007C20FF3CB
:1047CE0008C210F3B10E0301116F020E126F2BEC23
:1047DE000DF0B10E0F6F020E106F1FEC09F0090EE7
:1047EE002E6F0EEC00F0000E0201085D02E1000ECD
:1047FE00075D3BE3000E085D02E1100E075D35E23A
:10480E00060E006E07C2C2F008C2C3F0005006E0EA
:10481E000001C237C291C337FF0FF9D77F0E0301D4
:10482E000F6F530E106F000E116F01EC09F0C2C026
:10483E00F5F2C3C0F6F2B10E0201F76F020EF86F79
:10484E00F7EC11F0B10E03010F6F020E106F1FEC9B
:10485E0009F08FEC0EF0C4C1F5F2C5C1F6F2C2C07C
:10486E00F7F2C3C0F8F270EC12F002013151550AA2
:10487E00D8A483D04451230AD8A47FD0C00E0301FC
:10488E000F6F510E106F000E116F01EC09F0BAECA4
:10489E0012F0CD0E0301016F000E026FCC0E036FEE
:1048AE00000E046FCB0E056F000E066F000E076F25
:1048BE00020E086F2D0E096F020E0A6F190E0B6F86
:1048CE00020E0C6F2E0E0D6F020E0E6F40EC18F0D6
:1048DE00CD0E0301016F000E026FCC0E036F000EA2
:1048EE00046FCB0E056F000E066F000E076F020EE3
:1048FE00086F2D0E096F020E0A6F190E0B6F020E46
:10490E000C6F2E0E0D6F020E0E6FA1EC18F0CDC0B7
:10491E00F5F2CCC0F6F2CBC0F7F200C2F8F22DC21F
:10492E00F9F219C2FAF22EC2FBF272EC19F0BE0EB7
:10493E0003010F6F530E106F000E116F01EC09F093
:10494E000B0E03010F6F020E106F1FEC09F02D0EF0
:10495E000F6F540E106F000E116F01EC09F01A0E4E
:10496E0003010F6F020E106F1FEC09F08FEC0EF0AB
:10497E000201316B0101FA6BFB6B310E0201F56F17
:10498E00020EF66F8B0EF76F000EF86FE6EC15F059
:10499E0000C0FAF101C0FBF1000E026E0150025C84
:1049AE0002E10050000870E25E0E03010F6F500E20
:1049BE00106F000E116F01EC09F00101206B216BDD
:1049CE00000E215D02E10F0E205D5EE2060E026E0C
:1049DE0020C100F021C101F0025005E00036009028
:1049EE000136FF0FFAD700C0C2F001C0C3F0C4C138
:1049FE00F5F2C5C1F6F200C0F7F201C0F8F270ECA4
:104A0E0012F04F0E03010F6F540E106F000E116F48
:104A1E0001EC09F0C2C0F5F2C3C0F6F2B10E02010C
:104A2E00F76F020EF86FF7EC11F0B10E03010F6F76
:104A3E00020E106F1FEC09F0090E2E6F0EEC00F037
:104A4E00C4C10FF3C5C110F31FEC09F08FEC0EF0CB
:104A5E00C4C1F5F2C5C1F6F2190E0201F76F000ED0
:104A6E00F86FA9EC10F0150E0B6E4B0E0C6EBE0E01
:104A7E000D6E0D2EFED70C2EFCD70B2EFAD7000086
:104A8E000101204B212B9CD71DEC1AF042EF1EF09A
:024A9E00FFD740
:1054A20010EE1DF0820E006E010E016EA00EF66E61
:0E54B2004E0EF76E000EF86EA1EC10F0120018
:104AA0000000000000000000000000000000000006
:104AB00000000000000000000000000000000000F6
:104AC00000000000000000000000000000000000E6
:104AD00000000000000000000000000000000000D6
:104AE00000000000000000000000000000000000C6
:104AF00000000000000000000000000000000000B6
:104B000000000000000000000000000000000000A5
:104B10000000000000000000000000000000000095
:104B200000000000000000004242420000424242F9
:104B3000844221000084422100E700000000E700D9
:104B40002142840000214284010204081020408098
:104B50008040201008040201AA55AA55AA55AA555A
:104B6000815A244242245A81005864040464580043
:104B70000C1222444422120C7E81A59191A5817EC3
:104B80007E8195A1A195817E20342AE1E12A3420FD
:104B900010F884828284F810985CB65F5FB65C98E7
:104BA00000000000000000000000009F0000000066
:104BB000000007000007000000247E24247E24005B
:104BC00000242A7F2A1200000043231008C4C200D8
:104BD00000768995626080000000090503000000EE
:104BE00000001824428100000000814224180000C7
:104BF0000014087F081400000010107C1010000042
:104C00000000109070000000001010101010100034
:104C10000000C0C000000000004020100804020096
:104C2000007EA19189857E0000848281FF808000C2
:104C30000082C1A19189860000428189898976001C
:104C40000030282422FF2000008F89898989710083
:104C5000007E9191919160000001E111090503002E
:104C600000768989898976000006898989493E000C
:104C70000000006666000000000000AC6C00000050
:104C800000000814224100000024242424242400CD
:104C90000000412214080000000201B109060000D2
:104CA000000000000000000000FE21212121FE0084
:104CB00000FF898989897600007E81818181420097
:104CC00000FF818181423C0000FF89898981810048
:104CD00000FF090909010100007E81819191F20024
:104CE00000FF08080808FF00008181FF81810000A3
:104CF00000408081817F010000FF1818244281005C
:104D000000FF80808080800000FF02040402FF001A
:104D100000FF04081020FF00007E818181817E0059
:104D200000FF090909090600007E8181A141BE003A
:104D300000FF09192949860000868989898971003F
:104D4000000101FF01010000007F808080807F0062
:104D5000003F408080403F00007F806060807F0097
:104D600000C324181824C300000708F0F008070047
:104D700000C1A1918985830000FF818100000000AE
:104D8000001516FC161500000000008181FF0000D0
:104D90000004020102040000008080808080800006
:104DA0000001020400000000002054545478000068
:104DB000007E484848300000003844444420000049
:104DC00000304848487E0000003C4A4A4A0C000037
:104DD00000107C1202040000000C5252523E0000EF
:104DE000007E100808700000000000447D400000B4
:104DF00000204040443D00000000FE20508800009C
:104E0000000082FE80800000007804180478000012
:104E1000007C080404780000003844444438000052
:104E2000007C14140800000000081414187C000012
:104E3000007C0804040800000048545424000000CA
:104E400000043E4440200000003C4040207C000024
:104E5000001C2040201C0000003C4030403C000072
:104E6000004428102844000000000C50503C000072
:104E7000004464544C440000000008364100000027
:104E8000000000FF000000000000004136080000A4
:104E90000000060909060000001038541010100028
:044EA000000000000E
:044EA400000000000A
:044EA8000000000006
:024EAC002E00D6
:024EAE002000E2
:024EB0002000E0
:014EB20000FF
:024EB300640099
:104EB5003753006B4F00AC4F00224F0001510025C6
:0E4EC5005000345100CD5000195300795400B4
:044ED30000000000DB
:044ED70000000000D7
:044EDB008C3D2500E5
:104EDF000D0A68656C6C6F2C2069206765742079EA
:094EEF006F7572204D73672100FC
:084EF80054454D505F4F4E0080
:094F000054454D505F4F46460038
:054F09004D73673D003F
:054F0E0044454D4F0079
:084F1300454550524F4D3D0091
:074F1B0053706565643D0061
:104F220020536F75726365203A2031384634364B10
:104F320032325F746573745F4D6178373132313963
:104F42005F34784D6174726963653878385F534FA6
:104F520046545F5350495F4C4D3333355F313631E0
:094F62003233302E63200D0A00E9
:104F6B00204469726563746F7279203A20433A5F0B
:104F7B004D696B726F435F4D657350726F6A6574E9
:104F8B00735F4D696B726F435F4D617837323139A7
:104F9B005F345F6D617472696365387838200D0A10
:014FAB000005
:104FAC002050726F6A6574203A2031384634364B83
:104FBC0032325F4D4158373231395F34785F4D6151
:104FCC00745F3878385F535049315F536F6674772C
:0F4FDC005F4C4D3333352E6D63707069720A0070
:104FEB00496E6974206574207465737420696E74DE
:104FFB006572727570742054696D6572312020383A
:10500B00207820313235206D73656320736F69749E
:0A501B00203220736563200D0A00A7
:105025002053616973697220756E206E6F757665A0
:105035006175204D73672061766563206C6520740A
:1050450065726D696E616C20766961203C4D736790
:095055003D787878783E0D0A00E0
:10505E0041666669636865204D6573736167657344
:10506E00203020E0203135202073746F636B657320
:10507E0020656E20454550524F4D20647520504995
:08508E0043313846200D0A00F1
:10509600696E697420534F4654205350492020525C
:1050A60043333D436C6B202C5243353D446F75743E
:1050B60020205243303D4353202D3E204D4178372A
:0750C6003231393A0D0A00F6
:1050CD004D6573736167657320656E20454550525C
:1050DD004F4D206176656320636465203A203C4521
:1050ED004550524F4D3D303E202E2E20E020313583
:0450FD00200D0A0078
:10510100204D6F64756C65204D6174726963652013
:105111003878382061766563204D4158373132390E
:10512100202B2063617074657572204C4D333335CB
:035131000D0A0064
:10513400204D6F64652054656D706572617475727D
:10514400652061766563203C54454D505F4F4E3E6B
:10515400206F75203C54454D505F4F46463E0D0A26
:01516400004A
:105165000D0A4F4B2C2054656D70657220697320B4
:105175004F4646210D0A5265746F75722061752080
:0F518500646973706C617920747874200D0A006E
:1051940020202020426F6E6E6520416E6E65652072
:1051A400323031372E426F6E6E652053616E7465F6
:0C51B4002E426967204269736F7573001A
:1051C000525443204D414A20617520666F726D61D3
:1051D000742020553B32383B31323B31363B303442
:0B51E0003B31393B353923200D0A001C
:1051EB00446973706C6179203C303132333435361D
:1051FB003738393E20737572206D6174726963653F
:0A520B0073204C656473200D0A0047
:105215004461746520267432202046696E20203250
:105225003031372F30312F30312030304830304D4C
:065235003030533D200063
:10523B00696E6974204144432045413020657420D8
:10524B002D565245463D322C3556207375722052E1
:06525B004132200D0A00A3
:1052610044617465202654322046696E203D203306
:10527100312F31322F31362032333A35393A3539FF
:06528100203D3E203A0032
:105287004461746520267431206465627574203228
:105297003031362F31322F33302032334835394DC4
:0652A700303053203D00F1
:1052AD00496E69742049324332203430304B687A6C
:1052BD0020706F7572205254432044533133303770
:0452CD00200D0A00A6
:1052D1000D0A436C6F636B20696E697469616C655B
:1052E10020696E20203D20202E2E2E20204B687A12
:0452F100200D0A0082
:1052F50020202020202020202020202020202020A9
:10530500202020202020446966666572656E6365ED
:04531500203D3E00F9
:10531900B02AB0426F6E6E6520414E4E454520322F
:0E532900303137206120546F7573B02AB00008
:10533700204D696B726F6320372E302E3020313845
:0A5347004634364B3232200D0A00C6
:105351000A0D4D6973652061206C2768657572655A
:0753610020525443203A00E2
:10536800436C656172204D6174726963652032789F
:07537800203878380D0A000F
:10537F002020456570726F6D204D736720616472D8
:06538F0065737365200048
:105395000D0A4F4B2C2054656D7065722069732082
:0653A5004F4E210D0A002D
:1053AB000D0A4368616E6765205370656564205410
:0353BB006F200060
:1053BE004E65772044533133303720446174652075
:0253CE003A00A3
:1053D00050726573656E746174696F6E203A200D4A
:0253E0000A00C1
:1053E2000A0D205254432055706461746564200D87
:0253F2000A00AF
:1053F4003031323334353637383941424344454607
:0E5404004453313330372044617465203A0040
:0E5412004461746520267431204E6F772000AF
:0D542000446966666572656E6365203D0037
:0C542D00204E65772054696D653A200020
:0B543900436F6D70746575723D2000BC
:0B544400303132333435363738390050
:0A544F00456570726F6D2023200088
:085459002054696D653A200042
:075461000D0A206D3D200043
:075468002070747320200086
:05546F002020202000B8
:055474002020202000B3
:055479002020202000AE
:05547E002020202000A9
:055483002E2E2E2E006C
:05548800203E3E200063
:05548D00203D3E3A0045
:05549200202020200095
:0454970054B03D00D0
:03549B002E2E00B2
:03549E00B0430018
:020000040030CA
:0D000100281E3CFF9980FF0FC00FE00F404C
:0200000400F00A
:100000005061676520576562203A207061756C66A3
:100010006A756A6F2E667265652E6672203A2020B8
:100020004A6F79657578204E6F656C2032303136B5
:10003000457420426F6E6E6520416E6E65652000CE
:1000400050696331384634364B323220204D696B6B
:10005000726F432050726F20372E302E30202020B8
:100060003136204D65736720656E20454550524FEF
:100070004D206465203634206361726163742E0004
:100080004A6575782064652063617220204153437E
:100090004949646520203020E0203132372020207B
:1000A0004142434445464748494A4B4C4D4E4F50C8
:1000B0005152535455565758595A2061626364003F
:1000C00065666768696A6B6C6D6E6F707172737468
:1000D000757778797A23242B2D5F5B5D26B03D20E0
:1000E00020426F6E6E6520416E6E65652032303144
:1000F0003720002020202020202020202020200029
:1001000031372020202020202020202020202000E7
:100110005241532000202020202020202020200099
:100120005A65726F002020202020202020202000EF
:1001300057616C6F75002020202020202020200097
:100140005269656E002020202020202020202000E1
:10015000456D707479002020202020202020200070
:100160004C656572200020202020202020202000C7
:100170005269656E200020202020202020202000B1
:100180007669646500202020202020202020200087
:100190005269656E00202020202020202020200091
:1001A0004E49422000202020202020202020200016
:1001B000456D707479002020202020202020200010
:1001C000456D707479002020202020202020200000
:1001D000456D7074790020202020202020202000F0
:1001E000456D7074790020202020202020202000E0
:1001F000456D7074790020202020202020202000D0
:10020000456D7074790020202020202020202000BF
:10021000456D7074790020202020202020202000AF
:10022000456D70747900202020202020202020009F
:10023000456D70747900202020202020202020008F
:10024000456D70747900202020202020202020007F
:10025000456D70747900202020202020202020006F
:10026000456D70747900202020202020202020005F
:10027000456D70747900202020202020202020004F
:10028000456D70747900202020202020202020003F
:10029000456D70747900202020202020202020002F
:1002A000456D70747900202020202020202020001F
:1002B000456D70747900202020202020202020000F
:1002C000456D7074790020202020202020202000FF
:1002D000456D7074790020202020202020202000EF
:1002E000456D7074790020202020202020202000DF
:1002F000456D7074790020202020202020202000CF
:10030000456D7074790020202020202020202000BE
:10031000456D7074790020202020202020202000AE
:10032000456D70747900202020202020202020009E
:10033000456D70747900202020202020202020008E
:10034000456D70747900202020202020202020007E
:10035000456D70747900202020202020202020006E
:10036000456D70747900202020202020202020005E
:10037000456D70747900202020202020202020004E
:10038000456D70747900202020202020202020003E
:10039000456D70747900202020202020202020002E
:1003A000456D70747900202020202020202020001E
:1003B000456D70747900202020202020202020000E
:1003C000456D7074790020202020202020202000FE
:1003D000456D7074790020202020202020202000EE
:1003E000456D7074790020202020202020202000DE
:1003F000456D7074790020202020202020202000CE
:00000001FF
